:100000000C94DF010C94FA010C949B040C9477047B
:100010000C94FA010C940E130C94FA010C94FA014E
:100020000C94FA010C94FA010C9451130C94FA01FB
:100030000C94FA010C94FA010C94FA010C94FA0154
:100040000C94FA010C94FA010C94FA010C94FA0144
:100050000C94FA010C94FA010C943A051D5A3440A0
:10006000E17A34406ABC344091ED34407D3F354004
:10007000A47035402DB23540F2D23540B6F335404C
:100080003F353640666636408D97364017D9364044
:10009000643B3740EE7C374014AE37409EEF37402C
:1000A000B0723840E926394021B03A4093183C40BC
:1000B000350060008000B0001D013D015A017A0149
:1000C0009701B901DA01F901160240026D028202BC
:1000D000A202EF023203B003F203AA03A703A403B0
:1000E000A1039E039B039803940391038D038A034A
:1000F000860382037E037B03770372036E036A0326
:10010000660361035D03580353034F034A0345032A
:1001100040033B03360330032B03260320031B035A
:1001200015030F030A030403FE02F802F202EC02B5
:10013000E602DF02D902D302CC02C602BF02B90234
:10014000B202AC02A5029E02970291028A028302C9
:100150007C0275026E02680261025A0253024C026E
:1001600045023E0237023002290222021B0215021A
:100170000E0207020002F901F201EC01E501DE01C5
:10018000D801D101CB01C401BE01B701B101AA015F
:10019000A4019E01980192018C01860180017A01DF
:1001A00074016E01680163015D01580152014D0146
:1001B000470142013D01380133012E01290124018B
:1001C0001F011A01150111010C0108010301FF00B3
:1001D000FB00F600F200EE00EA00E600E200DE00BE
:1001E000DB00D700D300CF00CC00C800C500C200A0
:1001F000BE00BB002F03390342034B0353035C03D0
:1002000064036C0373037B03820388038F039503EA
:100210009B0326031C0312030703FD02F202E702FD
:10022000DC02D002C502B902AD02A1029502890228
:100230007C027002630257024A023E023202250229
:1002400019020C020002F401E801DC01D001C40132
:10025000B801AD01A20196018C01810176016C010A
:10026000620158014E0144013B0132012901200184
:1002700017010F010701FF00F700F000E900E1009E
:10028000DB00D400CD00C700C100BB00510A802AAA
:100290000000000A510A000059551801111E111BD7
:1002A000500B411B411F1101511F511B0000000049
:1002B00000000000000000000000510F91394114BF
:1002C0009131411E410E411D500F8020101548866E
:1002D0004014780570855115510E5195518E21901D
:1002E00081205015484450C528C0282009500000DE
:1002F000000000000000000054494D4552004155E7
:10030000544F00445249004D414E00534554004F54
:100310005054494F4E00445354415254004D53548D
:100320004F50004D53544152540041535441525484
:100330000053484F4F54005741495400434F554EC6
:10034000540044434F554E540042555A5A455200AA
:100350004F4E004F464600434C49434B004F4E0022
:100360004F4646004C4544004F4646004F4E004C19
:1003700049474854004155544F0054454D500000E2
:100380000102030405040500010203040502030041
:100390000159594D4D4444004D4D44445959004470
:1003A000444D4D5959003234480031324800313201
:1003B00048003234480032344800313248001124B9
:1003C0001FBECFEFD4E0DEBFCDBF11E0A0E0B1E0B3
:1003D000E6E8FAE202C005900D92AE33B107D9F714
:1003E00011E0AEE3B1E001C01D92A63BB107E1F719
:1003F0000C9436070C94000040E050E08B9A839AEE
:1004000080917A00806880937A0080917A0080647D
:1004100080937A0080917A0084FFFCCF30E0809155
:100420007A00806480937A0080917A0084FFFCCF08
:1004300020917800809179009927982F8827820F42
:10044000911D480F591F3F5F383048F38B988398B0
:1004500080917A008F7780937A00CA0123E0959586
:1004600087952A95E1F7089580937C0083E880932F
:100470007A000E94FC0108959F92AF92BF92CF92A2
:10048000DF92EF92FF920F931F93CF93DF93C0E021
:10049000D0E099240E94FC019C0180917C0088237B
:1004A00009F09DC080910001833009F04CC083E0C9
:1004B0002B3238078CF0AE01FA01EC50FE4F8591DB
:1004C00094918217930730F493944E5F5F4F99E1B4
:1004D000991590F76DE216C0E3E020323E078CF4E8
:1004E000AE01FA01EE5EFD4F859194912817390710
:1004F00030F493944E5F5F4FF3E6F91590F76BE29B
:1005000001C060E281E00E948806892D0E94FB0301
:100510009FE0A92EA82220E3A20E182F12951F708B
:10052000120F60E280E00E948806612F82E00E9444
:1005300088066A2D83E00E9488066AE284E00E94B1
:10054000880663E447C0843009F049C1E92DFF27DC
:10055000EE0FFF1FE652FF4F85919491821793078C
:1005600020F093948DE8891588F7892D0E940C045A
:10057000EC0193E6991560F46BE280E00E94880636
:100580008D2F992787FD9A95182F105D612F05C033
:1005900060E280E00E9488066BE281E00E948806AB
:1005A0000FE0A02EAC22E0E3AE0E14E0D595C79587
:1005B0001A95E1F78C2F8F708E0F682F82E00E94C2
:1005C00088066A2D83E00E9488066AE284E00E9421
:1005D000880666E485E00E94880660E0FDC08091A0
:1005E0007C00813009F0BFC0E90182E00E94340242
:1005F0000E94FC019C0140E050E0FA01E055FF4FF1
:10060000859194918217930730F493944E5F5F4FD6
:10061000F6E1F91590F7992029F486EF98E2A4E322
:10062000B0E419C025E1291528F48AEB99E4ACE37C
:10063000B0E411C0292D3327220F331F220F331F9F
:10064000245A3F4FF901E590F490F9013296059153
:100650001491D801C7018093010190930201A093E6
:100660000301B0930401A1E09A2E90927C00CE0188
:10067000AA2797FDA095BA2FBC01CD010E948F1427
:100680007B018C018091010190910201A0910301F5
:10069000B09104019C01AD01C801B7010E94E414AE
:1006A000DC01CB0120E030E040E85AE3BC01CD01A1
:1006B0000E94E414DC01CB0120E030E040EC50E487
:1006C000BC01CD010E94E4147B018C010E947214D4
:1006D0005B016C01862F9927AA2797FDA095BA2F59
:1006E000BC01CD010E948F14DC01CB019C01AD0146
:1006F000C801B7010E942F14DC01CB0120E030E0DB
:1007000048EC52E4BC01CD010E94E414DC01CB01B1
:10071000BC01CD010E9472147B018C018A2D0E94C4
:10072000FB03FFE0AF2EA822F0E3AF0E8E2D0E9458
:10073000FB03182F12951F70105D60E280E00E948D
:10074000880660E2892D0E94880660E282E00E94AD
:1007500088066A2D83E00E94880666E584E00E9490
:100760008806612F37CFC0917C00C230C1F58091DF
:1007700079000E94FB0380917800982F9F70E0E33E
:10078000AE2EA90E29E32A1518F477E3A72EA90E99
:10079000682F62956F70162F105D1A3308F0195F7D
:1007A00061E4892D0E94880664E481E00E94880645
:1007B00063E48C2F0E94880680917900805D682F09
:1007C00083E00E948806612F84E00E9488066A2DDB
:1007D00085E00E948806692D86E00E948806DF91E8
:1007E000CF911F910F91FF90EF90DF90CF90BF902E
:1007F000AF909F900895282F80E02A3018F08F5FE7
:100800002A50FBCF992734E0880F991F3A95E1F7DA
:10081000282B822F9927089520E030E0843620F09D
:100820002F5F3F4F8456FACF54E0220F331F5A9563
:10083000E1F78A3020F02F5F3F4F8A50FACF44E033
:10084000220F331F4A95E1F79927822B932B0895A6
:10085000209A229A239A259A85B1806D85B91DB870
:100860008EB18C608EB98CE080936B0080ED8093AC
:100870006C0080EC8CBB8DBB0E94C813809355012B
:10088000089523B12095207D8CB180958C70282B04
:10089000822F992786FF02C094E00FC027FF02C075
:1008A00095E00BC082FF02C093E007C083FF02C047
:1008B00092E003C084FF16C091E08091400188233C
:1008C00089F080913E01882359F490933F0181E0A3
:1008D00080933E0180914A01882311F00E941514F3
:1008E0001092400180EC8CBB10924C0108951F9235
:1008F0000F920FB60F9211242F933F934F935F9354
:100900006F937F938F939F93AF93BF93EF93FF93D7
:100910000E944104FF91EF91BF91AF919F918F9100
:100920007F916F915F914F913F912F910F900FBEEB
:100930000F901F9018951F920F920FB60F921124CF
:100940002F933F934F935F936F937F938F939F93D7
:10095000AF93BF93EF93FF930E944104FF91EF91F8
:10096000BF91AF919F918F917F916F915F914F91C7
:100970003F912F910F900FBE0F901F901895F894F4
:1009800080913E01882321F080913F0110923E0129
:10099000789499270895F999FECFF89492BD81BD76
:1009A000F89A789480B599270895F999FECFF8942C
:1009B00092BD81BD60BDFA9AF99AF999FECF7894FB
:1009C000089581118FEFE7E5F1E093E18193915074
:1009D00097FFFCCF089580E00E94E1048FE08093B0
:1009E000E70087EB8093E50087E08093E60080ECEA
:1009F0008093E4008091E40088608093E40010928A
:100A000046010895E82F20E030E0663090F58A52E4
:100A1000813558F4E13608F0EF7DEA52FF27EE0FFA
:100A2000FF1FE457FD4F25913491862F992780FFB2
:100A300002C05FE001C050EF6695E62FFF27E95A3C
:100A4000FE4FBC016170707043E0922F9F7084E094
:100A5000369527958A95E1F76115710511F0929504
:100A6000907F80818523892B80833596415047FF75
:100A7000ECCF08951F920F920FB60F921124DF92C0
:100A8000EF92FF920F931F932F933F934F935F9398
:100A90006F937F938F939F93AF93BF93CF93EF9376
:100AA000FF93DD2480914001882361F48091470108
:100AB0008F5F80934701843028F081E0809340016C
:100AC000D092470180914901833071F480914801AF
:100AD0008F5F80934801813148F081E08093490124
:100AE0008FE08093480102C0109248018091050177
:100AF00081508093050190915601992371F08823CC
:100B000071F480914501882321F481E080934601AE
:100B100006C081508093450102C090938401FF2458
:100B200090914601913009F06CC08091440185306C
:100B300010F4EF2C01C0E92EC0E000E010E080913D
:100B40008401992787FD9095800F911F97FD17C00D
:100B5000FF20A9F480918401992787FD9095F801E1
:100B6000E559FE4FE80FF91F8081DF2C87FF02C097
:100B700091E0D92E8F7721F4FC2EF39401C080E20E
:100B8000DD2029F0EE2019F06C2F80E201C06C2FDF
:100B90000E940205CF5F0F5F1F4FC63080F2ACEEA0
:100BA000B0E0E7E5F1E0C3E181918D93C150C7FF6B
:100BB000FBCF80914301811181E08093F40080910B
:100BC00042019091F900882311F0916001C09E7F4D
:100BD0009093F900809141019091EE00882311F0EB
:100BE000906201C09F7D9093EE0081E0F81611F4B1
:100BF0008AEF03C0809184018F5F809384011092FB
:100C0000460180910501882319F483E08093050152
:100C1000809144018A3019F41092440103C08F5F1F
:100C200080934401FF91EF91CF91BF91AF919F913C
:100C30008F917F916F915F914F913F912F911F9174
:100C40000F91FF90EF90DF900F900FBE0F901F90CD
:100C50001895FC01809146018823E1F7982F849133
:100C6000882391F0AF01ABE6B1E09F01F9018491D7
:100C70008D939F5F2F5F3F4F4F5F5F4FFA018491CE
:100C8000882311F0993190F3E92FFF27E559FE4FA2
:100C90001082973048F081E08093560110928401D1
:100CA00083E08093450104C01092560110928401A4
:100CB00081E0809346010895DC01E0914601EE2336
:100CC000E1F79E2F8C91882359F0FD01ABE6B1E04E
:100CD00081918D939F5F8081882311F09931C0F3BA
:100CE000E92FFF27E559FE4F1082973048F081E049
:100CF000809356011092840183E08093450104C0E3
:100D0000109256011092840181E08093460108956B
:100D1000893128F4E82FFF27E559FE4F60830895B5
:100D200090E2EBE6F1E088E19193815087FFFCCF00
:100D30000895809343010895909146019923E1F726
:100D40006093560190938401809346010895109218
:100D50004401089501972FEF8F3F920731F02CE760
:100D60000000215027FFFCCFF5CF0895CF93C0E0BE
:100D700080E88093610083E080936100C0937000FD
:100D800088E08093B60088EC8093B300C0936E0037
:100D900081E0809381008093B0008091B600282F7D
:100DA0003327217030708091B6009927847090703D
:100DB000282B392B232B89F788EE93E00E94AA0673
:100DC0004FEF51E0F89446BB47BB1092850010925C
:100DD00084001092B200B99BFECF109281007894EB
:100DE000B09B03C02FEF3FEF0AC090918400809129
:100DF0008500282F3327322F2227290F311D88E124
:100E00002B36380724F080916600815006C0285E9A
:100E1000374134F4809166008F5F8093660001C093
:100E2000C1E050938100CC2369F2CF9108950E94D4
:100E3000B60690E89093610083E08093610090BFD4
:100E400087E080937F008FE085B980EF8EB9259A87
:100E50002D9A0E9428040E94090F0E9439138CE0E9
:100E600090E00E94F4130E94EB040895CFEFD4E0C9
:100E7000DEBFCDBF0E941707789482E080937C008C
:100E80000E9434020E94FC0110928E0180E090E0EA
:100E90000E94CB04992790938601809385018F3F10
:100EA000910521F4109286011092850181E090E075
:100EB0000E94CB04992790939C0180939B018F3FC4
:100EC000910521F410929C0110929B0182E090E028
:100ED0000E94CB04992790938D0180938C018F3FC2
:100EE000910521F410928D0110928C0183E090E025
:100EF0000E94CB04992790939401809393018F3F94
:100F0000910521F4109294011092930184E090E0F5
:100F10000E94CB04992790938A01809389018F3F87
:100F2000910521F410928A011092890185E090E0E8
:100F30000E94CB0480938B018F3F11F410928B01A0
:100F400080918B0180934A0186E090E00E94CB045F
:100F5000992790939601809395018F3F910521F4F5
:100F6000109296011092950187E090E00E94CB04C8
:100F700080939F018F3F11F410929F0188E090E0D1
:100F80000E94CB04992790938801809387018F3F1B
:100F9000910521F4109288011092870189E090E078
:100FA0000E94CB0499279093900180938F018F3FEB
:100FB000910531F488E090E09093900180938F0147
:100FC0008AE090E00E94CB0499279093920180934D
:100FD00091018F3F910531F481E090E0909392016F
:100FE000809391010E9426140E94BF04E82E8091F4
:100FF0004C0190914D014E9720F088E18093600064
:10100000FFCF8091950190919601009709F42B9A5A
:101010008130910509F42B98029781F482E0809346
:101020007C000E9434020E94FC0123E0893E92076A
:101030000CF02B98885D93400CF42B9A209195012D
:10104000309196012330310579F4EE2021F0309370
:10105000A1012093A0018091A0019091A101892B71
:1010600011F02B9801C02B9A60918E01662369F4D0
:1010700088EF92E00E94290654E0E51609F4A5C61F
:1010800085E0E81609F0C0C6DBC16A3099F460E07B
:101090008EEF92E00E94290624E0E21609F495C63C
:1010A00045E0E41609F468C052E0E51609F0ACC664
:1010B0008BE091C6623399F460E083E093E00E9494
:1010C000290684E0E81609F4BBC125E0E21609F41C
:1010D000A5C142E0E41609F097C683E37CC66431FB
:1010E00091F460E087E093E00E94290654E0E51661
:1010F00009F442C085E0E81609F4C2C422E0E21611
:1011000009F082C691C16E3191F460E08BE093E00A
:101110000E94290644E0E41609F480C155E0E51672
:1011200009F453C682E0E81609F06EC6A4C468321A
:10113000C9F460E08FE093E00E94290624E0E21603
:1011400009F49EC445E0E41609F47AC152E0E516BC
:1011500009F447C681E0E81609F056C688E1809395
:101160006000FFCF633381F560E086E193E00E9489
:10117000290623E0E21611F482E32DC641E0E416CD
:1011800009F042C6109288011092870181E090E038
:10119000909392018093910125E320938E012091F9
:1011A0008F01309190013093980120939701909393
:1011B0009A01809399019093A4018093A301909345
:1011C0009E0180939D0165C1653309F097C02A98FF
:1011D00081E00E9499068091990190919A0101976E
:1011E00041F484EF91E00E94AA0610929A011092B5
:1011F000990110924D0110924C012091A301309160
:10120000A4012330310559F43093A1012093A001AA
:1012100080919F01882319F081EC80938000223017
:10122000310519F41092800020C0232BF1F4809135
:10123000970190919801019790939801809397015D
:10124000892B41F42A9A83E380938E0180E00E94E7
:1012500099060BC086E380938E0180919101909155
:1012600092019093A4018093A3012091A301309156
:10127000A401C9016CE370E00E942F15FB01C901B4
:101280006CE370E00E942F158C018E2F0E94FB03EF
:10129000C82F7FE0F72EF82250E3F50EC295CF70ED
:1012A000C50F802F0E94FB03082F182F1F70105DA1
:1012B00002950F70005D63E580E00E94880660E2A1
:1012C00081E00E9488066C2F82E00E9488066F2DC4
:1012D00083E00E948806602F84E00E948806612FC8
:1012E00085E00E94880660E086E00E94880683E030
:1012F000E81609F089C52A9A83E3C2C1663309F06A
:1013000070C02A9A10924D0110924C018091A30155
:101310009091A401892BA9F485E380938E0180919B
:101320009D0190919E01880F991F01969093A401B1
:101330008093A301019790939E0180939D010E9449
:101340003913E091A301F091A401E330F10521F4F8
:10135000F093A101E093A001CF016CE370E00E9443
:101360002F159B01CF016CE370E00E942F158C01BB
:10137000822F0E94FB03C82F6FE0F62EF82220E395
:10138000F20EC295CF70C20F802F0E94FB03082F70
:10139000182F1F70105D02950F70005D67E580E0EB
:1013A0000E94880660E281E00E9488066C2F82E03D
:1013B0000E9488066F2D83E00E948806602F84E0DB
:1013C0000E948806612F85E00E94880660E086E022
:1013D0000E94880643E0E41609F016C52A9A82E3C3
:1013E0004FC1663179F460E08DE193E00E942906F7
:1013F0002A9A53E0E51691F081E0E81609F004C559
:1014000085E1E9C4653191F460E083E293E00E94F4
:1014100029062A9823E0E21619F42A9A84E1DBC40B
:1014200041E0E41609F0F0C486E1D5C46B30A1F5C3
:1014300060E08AE293E00E94290653E0E51611F489
:101440008AE0C9C481E0E81609F0DEC48CE080932C
:101450008E018091890190918A01909398018093E7
:10146000970120919B0130919C018CE390E0289F93
:10147000A001299F500D389F500D112480918501A6
:1014800090918601840F951F01969093A4018093FB
:10149000A3010E943913B8C46C3009F077C02A98B0
:1014A00081E00E94990610924D0110924C0120910A
:1014B000A3013091A4012330310559F43093A101E7
:1014C0002093A00180919F01882319F081EC8093E3
:1014D00080002230310519F4109280002FC0232B98
:1014E00069F58091970190919801019790939801E7
:1014F00080939701892B41F42A9A8BE080938E0187
:1015000080E00E9499061AC08DE080938E012091A0
:101510009301309194018CE390E0289FA001299FD2
:10152000500D389F500D112480918C0190918D01A8
:10153000840F951F9093A4018093A3012091A30190
:101540003091A401C9016CE370E00E942F15FB01EA
:10155000C9016CE370E00E942F158C018E2F0E9450
:10156000FB03C82F5FE0F52EF82250E3F50EC2957D
:10157000CF70C50F802F0E94FB03082F182F1F70FC
:10158000105D02950F70005D63E559C06D3009F084
:101590007DC02A9A10924D0110924C018091A301B6
:1015A0009091A401892BE9F48CE080938E01209125
:1015B0009B0130919C018CE390E0289FA001299F22
:1015C000500D389F500D1124809185019091860116
:1015D000840F951F01969093A4018093A3010E940C
:1015E0003913E091A301F091A401E330F10521F456
:1015F000F093A101E093A001CF016CE370E00E94A1
:101600002F159B01CF016CE370E00E942F158C0118
:10161000822F0E94FB03C82F4FE0F42EF82250E3E4
:10162000F50EC295CF70C50F802F0E94FB03082FC7
:10163000182F1F70105D02950F70005D67E580E048
:101640000E94880660E281E00E9488066C2F82E09A
:101650000E9488066F2D83E00E948806602F84E038
:101660000E948806612F85E00E94880660E086E07F
:101670000E94880683E0E81609F0C6C32A9A8BE028
:1016800080938E0180E00E949906BEC36F31B9F449
:1016900060E081E393E00E94290624E0E21609F469
:1016A000D0C145E0E41609F4C7C153E0E51609F4DA
:1016B000E7C182E0E81609F0A7C381E28CC361327A
:1016C00009F051C081E00E94990681E080934101B8
:1016D00024E0E21631F48091850190918601019613
:1016E00008C045E0E41649F4809185019091860197
:1016F0000197909386018093850180918501909157
:101700008601CC9734F08BE390E090938601809330
:101710008501809185019091860197FF04C0109208
:101720008601109285018E2D8250823058F482E21B
:1017300080938E01109241016091850180E090E0DC
:101740000E94D50451E0E51609F062C08FE1809354
:101750008E0180E00E9499061092410160918501FE
:1017600080E090E053C0623209F06CC081E00E94DA
:10177000990681E08093420124E0E21631F48091E1
:101780009B0190919C01019608C045E0E41649F444
:1017900080919B0190919C01019790939C01809373
:1017A0009B0180919B0190919C018436910534F0BE
:1017B00083E690E090939C0180939B0180919B0134
:1017C00090919C0197FF04C010929C0110929B0184
:1017D0008E2D8250823058F481E280938E011092D7
:1017E000420160919B0181E090E00E94D50451E0AC
:1017F000E51671F48FE180938E0180E00E949906D6
:101800001092420160919B0181E090E00E94D5041A
:1018100080919B010E94FB03C82F3FE0F32EF8222A
:1018200080E3F80EC295CF70C80F809185010E94A9
:10183000FB03082F182F1F70105D02950F70005DBD
:1018400063E586C06032B9F460E087E393E00E940C
:10185000290624E0E21609F40EC145E0E41609F475
:1018600005C153E0E51609F40BC182E0E81609F062
:10187000CBC283E2B0C2633209F07FC081E00E9434
:10188000990681E08093410124E0E21631F48091D1
:101890008C0190918D01019608C045E0E41649F451
:1018A00080918C0190918D01019790938D0180938F
:1018B0008C0180918C0190918D01CC9734F08BE359
:1018C00090E090938D0180938C0180918C01909198
:1018D0008D0197FF04C010928D0110928C018E2D06
:1018E0008250823058F484E280938E01109241013C
:1018F00060918C0182E090E00E94D50451E0E516F1
:1019000071F480E280938E0180E00E94990610922B
:10191000410160918C0182E090E00E94D5048091A9
:1019200093010E94FB03C82F2FE0F22EF82280E3E0
:10193000F80EC295CF70C80F80918C010E94FB03F6
:10194000082F182F1F70105D02950F70005D67E55E
:1019500080E00E94880660E281E00E9488066C2F89
:1019600082E00E9488066F2D83E00E948806602F27
:1019700084E00E948806612F24C1643209F052C0BD
:1019800081E00E94990681E08093420124E0E21602
:1019900031F48091930190919401019608C045E043
:1019A000E41649F4809193019091940101979093EA
:1019B00094018093930180919301909194018436D6
:1019C000910534F083E690E0909394018093930125
:1019D000809193019091940197FF04C0109294011B
:1019E000109293018E2D8250823058F483E28093BE
:1019F0008E01109242016091930183E090E00E9479
:101A0000D50451E0E51609F08ACF80E280938E017B
:101A100080E00E949906109242016091930183E058
:101A200090E07BCF6532C1F460E08CE393E00E94EC
:101A3000290624E0E21611F480E2CDC145E0E41667
:101A400011F487E3C8C153E0E516D1F082E0E8164F
:101A500009F0DAC186E2BFC16733D1F460E082E405
:101A600093E00E94290624E0E21611F485E2B3C156
:101A700045E0E41611F48FE1AEC153E0E51611F430
:101A80008EE1A9C182E0E81609F0BEC188E3A3C1D6
:101A90006632D9F524E0E21631F480918901909103
:101AA0008A01019608C045E0E41649F48091890155
:101AB00090918A01019790938A0180938901809186
:101AC000890190918A018436910534F083E690E093
:101AD00090938A01809389018091890190918A0174
:101AE00097FF04C010928A011092890151E0E51617
:101AF00049F485E280938E016091890184E090E051
:101B00000E94D504809189013CC0683309F061C00E
:101B100024E0E21631F480918F01909190010196BA
:101B200008C045E0E41649F480918F01909190013E
:101B300001979093900180938F0180918F019091F4
:101B400090010A9734F089E090E090938A018093A5
:101B500089018091890190918A0197FF04C01092B8
:101B60008A011092890151E0E51649F487E38093D8
:101B70008E0160918F0189E090E00E94D5048091F0
:101B80008F010E94FB03C82F9FE0F92EF82280E30B
:101B9000F80EC295CF70C80F63E480E00E948806FB
:101BA00060E281E00E94880660E282E00E9488068E
:101BB00060E283E00E9488066C2F84E00E94880621
:101BC0006F2D85E00E94880660E086E00E9488060E
:101BD0001BC16932B9F460E089E493E00E942906F0
:101BE00023E0E21609F4F1C042E0E41611F48AE2BF
:101BF000F2C055E0E51609F486C084E0E81609F065
:101C000003C17BC06A3221F560919F01662321F0F8
:101C100060E080E593E002C083E593E00E9429063E
:101C200023E0E21649F489E280938E0160919F01DE
:101C300087E090E00E94D5044CEFE40E51E05E1581
:101C400008F4E2C080919F01852780939F01DCC04A
:101C50006B32B9F460E087E593E00E94290683E0E7
:101C6000E81609F4B2C022E0E21611F48CE2B3C027
:101C700045E0E41609F4BAC054E0E51609F0C4C022
:101C8000B0C06C3239F560918B01662321F060E0C1
:101C90008DE593E002C080E693E00E94290683E090
:101CA000E81661F48BE280938E0180918B01809322
:101CB0004A01682F85E090E00E94D5042CEFE20EE7
:101CC00041E04E1508F4A0C080918B0184278093D9
:101CD0008B019AC06D32C9F460E084E693E00E9403
:101CE000290653E0E51609F470C082E0E81611F405
:101CF0008EE271C025E0E21611F48FE26CC044E080
:101D0000E41609F081C08BE266C06E3209F053C060
:101D10002115310521F460E088E693E014C02130FC
:101D2000310521F460E08CE693E00DC022303105EE
:101D300021F460E08FE693E006C02330310529F4FA
:101D400060E085E793E00E94290653E0E51651F430
:101D50008DE280938E016091950186E090E00E9473
:101D6000D50452C085E0E81689F4809195019091E0
:101D700096010196909396018093950104970CF437
:101D800043C010929601109295013EC024E0E216E5
:101D9000D9F58091950190919601019790939601C4
:101DA0008093950197FF30C083E090E09093960177
:101DB0008093950129C06F32D9F460E08AE793E0FF
:101DC0000E94290643E0E41611F488E204C052E0C0
:101DD000E51621F480E380938E0116C085E0E816B5
:101DE00011F489E2F8CF24E0E21671F48DE2F3CF2A
:101DF000603351F443E0E41619F48FE280938E01CE
:101E000010927C000E943C0260E081E00E949C06EF
:101E1000EBC888EE93E00E94AA06F89480917000C7
:101E20008E7F8093700088E08093B6001092B2009D
:101E30008091B00085608093B0008091B600282F1B
:101E40003327217030708091B6009927847090708C
:101E5000282B392B232B89F78FEF87BB80917000BC
:101E600081608093700078941092A4011092A30175
:101E70001092A9018CE08093A2018BE18093A501CF
:101E800088E08093A80184E090E09093A70180937C
:101E9000A6010895DF92EF92FF920F931F93CF93C5
:101EA00080911301882341F48091A201E82FFF273C
:101EB000EC5EFE4F808102C08091A2010E94FB0374
:101EC000C82F2FE0D22ED82280E3D80EC295CF7033
:101ED000C80F8091A9010E94FB03082F9FE0E92E03
:101EE000E82280E3E80E02950F70080F8091A301AD
:101EF0000E94FB03182F8FE0F82EF12280E3F80EEA
:101F000012951F70180F6C2F80E00E9488066D2DAF
:101F100081E00E948806602F82E00E9488066E2D74
:101F200083E00E948806612F84E00E9488066F2D5E
:101F300085E00E94880660E086E00E94880681E0D5
:101F40000E94990660E081E00E949C0680E090E09B
:101F5000CF911F910F91FF90EF90DF900895CF9256
:101F6000DF92EF92FF920F931F93CF93C82E809131
:101F70003901882361F08091A20180934E01809104
:101F8000A90180934F018091A3018093500180911A
:101F90001301882341F480914E01E82FFF27EC5E66
:101FA000FE4F808102C080914E010E94FB03C82F2A
:101FB0005FE0F52EF82280E3F80EC295CF70C80FCF
:101FC00080914F010E94FB03182F4FE0E42EE8227E
:101FD00080E3E80E12951F70180F809150010E9447
:101FE000FB03082F3FE0D32ED82280E3D80E0295C2
:101FF0000F70080F6C2F772780915101882309F407
:10200000606880E00E9488066F2D772780915101DB
:10201000882309F4606881E00E948806612F772791
:1020200080915101813009F4606882E00E94880645
:102030006E2D772780915101813009F4606883E02B
:102040000E948806602F772780915101823009F421
:10205000606884E00E9488066D2D77278091510189
:10206000823009F4606885E00E94880660E086E0BE
:102070000E94880681E00E949906CC2011F00E94FF
:10208000A70660E081E00E949C0681E08093390110
:1020900084E0C81649F480915101E82FFF27E25BE4
:1020A000FE4F80818F5F0BC085E0C81651F4809190
:1020B0005101E82FFF27E25BFE4F80818150808332
:1020C0002CC083E0C81641F480915101882311F49B
:1020D00082E00AC0815008C082E0C81641F48091B5
:1020E00051018230C1F08F5F8093510116C081E0B1
:1020F000C81699F4F89480914E018093A2018091C2
:102100004F018093A9018091500199279093A401D8
:102110008093A30178941092510180914E018F3FDA
:1021200019F487E180934E0180914E01883110F0BF
:1021300010924E0180914F018F3F19F48BE38093F1
:102140004F0180914F018C3310F010924F0180911C
:1021500050018F3F19F48BE380935001809150011F
:102160008C3310F0109250011092390180E090E011
:10217000CF911F910F91FF90EF90DF90CF90089536
:10218000CF93C82F80913A01882371F010923A01C1
:1021900060911301613019F486EA93E003C061E0B5
:1021A0008AEA93E00E942906C43081F46091130109
:1021B000613029F4109213018EEA93E019C081E096
:1021C00080931301682F82EB93E012C0C53099F41D
:1021D00080911301882339F481E080931301682FE3
:1021E00086EB93E005C01092130161E08AEB93E067
:1021F0000E94290604C0C13011F4C0933A0180E066
:1022000090E0CF910895AF92BF92CF92DF92EF927C
:10221000FF920F931F938091A6010E94FB03F82E5B
:10222000EFE0CE2EC82280E3C80EF694F694F69422
:10223000F694F80E8091A8010E94FB03E82E7FE03F
:10224000B72EB82280E3B80EE694E694E694E694BE
:10225000E80E8091A5010E94FB03D82E6FE0A62E08
:10226000A82280E3A80ED694D694D694D694D80EFD
:1022700080914B01E82FFF2707E011E0EE0FFF1FD1
:10228000E00FF11F0190F081E02D84916F2D0E94ED
:10229000880680914B01E82FFF27EE0FFF1FE00F0C
:1022A000F11F0190F081E02D319684916C2D0E94F8
:1022B000880680914B01E82FFF27EE0FFF1FE00FEC
:1022C000F11F0190F081E02D329684916E2D0E94D5
:1022D000880680914B01E82FFF27EE0FFF1FE00FCC
:1022E000F11F0190F081E02D339684916B2D0E94B7
:1022F000880680914B01E82FFF27EE0FFF1FE00FAC
:10230000F11F0190F081E02D349684916D2D0E9493
:10231000880680914B01E82FFF27EE0FFF1FE00F8B
:10232000F11F0190F081E02D359684916A2D0E9475
:10233000880660E086E00E94880681E00E94990697
:1023400060E081E00E949C0680E090E01F910F9188
:10235000FF90EF90DF90CF90BF90AF900895FF92E5
:102360000F931F93CF93F82E80913B01882361F048
:102370008091A601809352018091A801809353011E
:102380008091A50180935401C0913C01CC23C9F4F4
:10239000809152010E94FB03182F082F0F70005DDF
:1023A00012951F70105D60E28C2F0E94880660E21B
:1023B00081E00E94880669E582E00E94880669E55E
:1023C00035C0C130C9F4809153010E94FB03182F1E
:1023D000082F0F70005D12951F70105D60E280E0A5
:1023E0000E94880660E28C2F0E9488066DE482E0DD
:1023F0000E9488066DE41AC0C23019F5809154011C
:102400000E94FB03182F082F0F70005D12951F709C
:10241000105D60E280E00E94880660E281E00E9438
:10242000880664E48C2F0E94880664E483E00E949E
:102430008806612F84E00E948806602F85E00E9454
:10244000880660E086E00E94880680E00E94990687
:10245000FF2011F00E94A70660E081E00E949C0628
:1024600081E080933B0184E0F81649F480913C01BF
:10247000E82FFF27EE5AFE4F80818F5F0BC085E06B
:10248000F81651F480913C01E82FFF27EE5AFE4FD9
:102490008081815080832CC083E0F81641F48091C4
:1024A0003C01882311F482E00AC0815008C082E018
:1024B000F81641F480913C018230C1F08F5F809327
:1024C0003C0116C081E0F81699F4F894809152010D
:1024D00099279093A7018093A6018091530180933F
:1024E000A801809154018093A501789410923C0139
:1024F000809152018F3F19F483E6809352018091BD
:102500005201843610F010925201809153018823B9
:1025100019F48CE080935301809153018D3018F0B1
:1025200081E0809353018091A8018230C9F4209109
:10253000A6013091A701C90183709070892B81F4A5
:10254000C90164E670E00E942F15892B39F4C90196
:1025500060E971E00E942F15892B11F4EDE107C0AD
:1025600080915301E82FFF27E45DFE4FE0818091C9
:102570005401882311F4E093540180915401E81729
:1025800018F481E08093540110923B0180E090E0C8
:10259000CF911F910F91FF900895CF93C82F8091F5
:1025A0003D01882379F010923D0180914B01E82F85
:1025B000FF27EE0FFF1FE35FFE4F61E080819181F7
:1025C0000E942906C43049F480914B01823018F0F2
:1025D00010924B010DC08F5F09C0C530B9F48091D6
:1025E0004B01882311F482E001C0815080934B019C
:1025F00080914B01E82FFF27EE0FFF1FE35FFE4F97
:1026000061E0808191810E94290604C0C13011F4EB
:10261000C0933D0180E090E0CF9108951F920F920A
:102620000FB60F9211248F939F938091A3019091E5
:10263000A40101979093A4018093A3018091A0012C
:102640009091A101009729F001979093A1018093A7
:10265000A00180914C0190914D01019690934D0104
:1026600080934C019F918F910F900FBE0F901F9000
:10267000189583E0EEEAF1E011921192815087FF04
:10268000FBCF9FEFEAEAF1E083E09193815087FF6F
:10269000FCCF82E080936E0086E287BD8CE084BD33
:1026A00008951F920F920FB60F9211240F931F934C
:1026B0002F933F934F935F936F937F938F939F934A
:1026C000AF93BF93CF93EF93FF93C3E00EEA11E074
:1026D000D801ED91FD918D01309709F00995C15018
:1026E000C7FFF6CFEAEAF1E0C3E080818F3F21F037
:1026F000882311F081508083C1503196C7FFF5CFF8
:10270000FF91EF91CF91BF91AF919F918F917F9169
:102710006F915F914F913F912F911F910F910F906A
:102720000FBE0F901F901895AC0120E0EEEAF1E08B
:10273000819191918417950761F02F5F2430C0F348
:1027400020E0EEEAF1E080819181892B29F4518328
:10275000408381E090E008952F5F3296243098F313
:1027600080E090E008959C0140E0EEEAF1E0808195
:1027700091818217930729F41182108281E090E001
:1027800008954F5F3296443090F380E090E00895D2
:1027900090E0E92FFF27E655FE4F80819F5F8F3F36
:1027A00021F41082892F99270895943090F380E0C6
:1027B00090E00895F894E82FFF27E755FE4F6083D7
:1027C00078940895F894E82FFF27E755FE4F80810D
:1027D000789499270895F894E82FFF27E755FE4F3E
:1027E0008FEF8083789408959C01832F992780939D
:1027F000C5002093C40082E08093C00080E18093F4
:10280000C10086E08093C2000895982F8091C00097
:1028100085FFFCCF9093C60008958091C000882367
:10282000E4F78091C60099270895CF93C9E02D9AC7
:1028300081E090E00E94AA062D9881E090E00E943D
:10284000AA06C150C7FFF3CFCF9108951092800020
:1028500089E08093810080E180938800089550583A
:10286000192E84D001D06AC0BA1762077307840793
:102870009507B1F188F40EF410940B2EBA2FA02D09
:10288000062E622F202D072E732F302D082E842F19
:10289000402D092E952F502DFF275523B9F0591B98
:1028A00049F0573E98F0469537952795A795F04003
:1028B0005395C9F776F0BA0F621F731F841F30F467
:1028C000879577956795B795F040939517FA0F2EF2
:1028D0000895BF1BBB27BA0B620B730B840BF6CF9B
:1028E000DEF670C097FB4ED09F3738F0FEE9F91B3B
:1028F000982F872F762F6B2F05C061C096958795EF
:1029000077956795F150D0F73EF490958095709546
:1029100061957F4F8F4F9F4F0895E89403C097FBB9
:102920000EF4F3DFB62F672F782F892F9EE900244E
:1029300005C09A95BB0F661F771F881F1124992326
:10294000A1F08823B2F79F3F59F0BB0F48F421F460
:10295000002011F460FF04C06F5F7F4F8F4F9F4FC7
:10296000881F9795879597F9089529C0052E092600
:1029700007FA440F551F5F3F79F0AA27A51708F003
:1029800051E04795880F991F9F3F31F0BB27B9173A
:1029900008F091E0879508959F919F9111245CC064
:1029A00097FB880F991F9F3F31F0BB27B91708F09D
:1029B00091E0879508959F919F9111244DC06627BE
:1029C0007727882799270895D1DF01D0B7CF99239A
:1029D00039F0552329F09F575F57950F13F49AF15B
:1029E000F1CF91589F3FE1F3629FA12D0F92BB273A
:1029F000639FA00DB11DEE27729FA00DB11DEE1FAC
:102A0000AF93AA27649FB00DE11D739FB00DE11D28
:102A1000AA1F6627829FB00DE11DA61F5527749F30
:102A2000E00DA11D551F839FE00DA11D561F849F22
:102A3000A00D511D852F7A2F6E2F1F900F90882388
:102A40001AF4939539F408C0000C111CBB1F661FC3
:102A5000771F881F012808959FEF80EC0895AA1B17
:102A6000BB1B51E107C0AA1FBB1FA617B70710F079
:102A7000A61BB70B881F991F5A95A9F780959095AB
:062A8000BC01CD01089528
:102A8600039A993940030F8B0385037F039F0398AD
:102A9600039103010C0102030405060708090A0B4A
:102AA6000C0102030405060708090A0B001F1C1F78
:0E2AB6001E1F1E1F1F1E1F1E1F0101010201F9
:00000001FF
